:100000000C9461000C9473000C9473000C947300B6
:100010000C9473000C9473000C9473000C94730094
:100020000C9473000C9473000C9473000C94730084
:100030000C9473000C9473000C9473000C94730074
:100040000C94F8000C9473000C9473000C947300DF
:100050000C9473000C9473000C9473000C94730054
:100060000C9473000C94730000000000240027001F
:100070002A000000000023002600290000000000E4
:10008000250028002B0004040404040404040202D4
:100090000202020203030303030301020408102007
:1000A0004080010204081020010204081020000012
:1000B0000008000201000003040700000000000027
:1000C000000011241FBECFEFD8E0DEBFCDBF21E07E
:1000D000A0E0B1E001C01D92AB30B207E1F70E9491
:1000E00042010C949F020C940000833081F028F4AC
:1000F000813099F08230A9F008958730A9F08830D6
:10010000C9F08430B1F4809180008F7D03C080916C
:1001100080008F7780938000089584B58F7784BDA9
:10012000089584B58F7DFBCF8091B0008F77809349
:10013000B00008958091B0008F7DF9CFCF93DF9309
:10014000282F30E0F901E255FF4F8491F901E6567E
:10015000FF4FD491F901EA57FF4FC491CC23A1F08E
:1001600081110E947500EC2FF0E0EE0FFF1FEE589A
:10017000FF4FA591B491EC91ED2381E090E009F45B
:1001800080E0DF91CF91089580E090E0FACFCF93A7
:10019000DF9390E0FC01E656FF4F24918A579F4F72
:1001A000FC0184918823D1F090E0880F991FFC0115
:1001B000E859FF4FA591B491FC01E458FF4FC59158
:1001C000D49161110EC09FB7F8948C91E22FE09505
:1001D0008E238C932881E223E8839FBFDF91CF9108
:1001E00008958FB7F894EC91E22BEC938FBFF6CF84
:1001F0001F920F920FB60F9211242F933F938F935C
:100200009F93AF93BF938091070190910801A091B4
:100210000901B0910A013091060123E0230F2D3727
:1002200058F50196A11DB11D209306018093070189
:1002300090930801A0930901B0930A0180910201F3
:1002400090910301A0910401B09105010196A11DB7
:10025000B11D8093020190930301A0930401B09318
:100260000501BF91AF919F918F913F912F910F9079
:100270000FBE0F901F90189526E8230F0296A11D20
:10028000B11DD2CF789484B5826084BD84B581607D
:1002900084BD85B5826085BD85B5816085BD809151
:1002A0006E00816080936E001092810080918100C9
:1002B00082608093810080918100816080938100C1
:1002C000809180008160809380008091B100846083
:1002D0008093B1008091B00081608093B0008091E4
:1002E0007A00846080937A0080917A0082608093A3
:1002F0007A0080917A00816080937A0080917A0000
:10030000806880937A001092C10060E082E00E94D1
:10031000C70060E083E00E94C70060E084E00E94C4
:10032000C70060E085E00E94C70060E086E00E94B0
:10033000C70061E089E00E94C700C4E6D0E09FE802
:10034000492E90E0592E20E0622E20E0722E09E125
:1003500010E032E3E32EF12C4BE4C42ED12C54E612
:10036000A52EB12C82E00E949E000197C1F483E08B
:100370000E949E00892B99F484E00E949E00892BA4
:1003800071F485E00E949E00892B49F486E00E946A
:100390009E00892B21F4109201011092000183E04C
:1003A0000E949E000197C1F482E00E949E00892B6A
:1003B00099F484E00E949E00892B71F485E00E94EC
:1003C0009E00892B49F486E00E949E00892B21F42F
:1003D000109301010093000184E00E949E000197A8
:1003E000C1F482E00E949E00892B99F483E00E9470
:1003F0009E00892B71F485E00E949E00892B49F4B0
:1004000086E00E949E00892B21F4F0920101E09287
:10041000000185E00E949E000197C1F482E00E94E5
:100420009E00892B99F483E00E949E00892B71F431
:1004300084E00E949E00892B49F486E00E949E0081
:10044000892B21F4D0920101C092000186E00E9424
:100450009E000197C1F482E00E949E00892B99F4CE
:1004600083E00E949E00892B71F484E00E949E002C
:10047000892B49F485E00E949E00892B21F4B092DB
:100480000101A0920001E7EBF0E08491E3EAF0E0E3
:100490002490F2013490332009F180900001909073
:1004A000010181110E947500E32DF0E0EE0FFF1FA6
:1004B000E458FF4F259134914FB7F894C401BE0121
:1004C0000E947702FFEFF69F602D1124F9018081D1
:1004D00061110BC02094282220824FBF6114710447
:1004E00009F440CF0E9400003DCF282AF5CF97FBAA
:1004F000072E16F4009407D077FD09D00E948B02D6
:1005000007FC05D03EF4909581959F4F0895709516
:1005100061957F4F0895AA1BBB1B51E107C0AA1F1D
:10052000BB1FA617B70710F0A61BB70B881F991F94
:100530005A95A9F780959095BC01CD010895F8943E
:02054000FFCFEB
:00000001FF
